:100000000C94DE010C94FB010C94FB010C94FB019D
:100010000C94FB010C94FB010C94FB010C94FB0170
:100020000C94FB010C94FB010C949D1F0C946F200D
:100030000C948F1A0C94FB010C94FB010C94FB01A3
:100040000C94FB010C94FB010C94FB010C94FB0140
:100050000C94FB010C94171B0C94FB010C94FB01FA
:100060000C94FB010C94FB010C94FB010C94FB0120
:100070000C94FB010C94FB010C94FB010C94FB0110
:100080000C94FB010C94FB010C94FB010C94FB0100
:100090000C94FB010C94FB010C94FB010C94FB01F0
:1000A0000C94FB010C94FB010C94FB01C404C404EC
:1000B000F004F004580576058E068E0681051A06B2
:1000C0002B062B06DC200321FB210321FB214F21E2
:1000D0007221FB21C921D82114001A000800150043
:1000E00017001C0018000C0012001300040016007A
:1000F000070009000A000B000D000E000F00290088
:100100001D611B64064319442A422C4105451174A4
:10011000107128721E001F00200021002200230001
:1001200024002500260027003A003B003C003D004B
:100130003E003F004000410042004300010001003A
:10014000010001004C00010001000100010001005C
:100150001E021F0220022102220223022402250283
:1001600026022702440045000100010001000100B1
:100170000100010001003500010001000100010043
:100180000100010001000100010001000100010067
:100190000100010001002D002E002F003000310071
:1001A0002B0001000100010001003600370038007B
:1001B00033003400010001000100010001000100D2
:1001C0005000510052004F000100010001000100E9
:1001D00001002D022E022F02300231022B000100FD
:1001E00001000100010036023702380233023402F6
:1001F0000100010001000100010001004A004E0061
:100200004B004D00B200B500B100B3000100010089
:100210000100010001004600010001000100010091
:100220000100010001000100BE5CBF5C0100010093
:1002300001000100005C010001000100010001005B
:10024000100347006800650072006B0069006E00D3
:1002500000002003340030002000500065007200D0
:10026000630065006E007400200043006C007500A0
:10027000620000000403090409023B00020100A01F
:10028000FA09040000010301010009211101000124
:100290002240000705810308000109040100010351
:1002A00000000009211101000122B60007058203A8
:1002B00020000112010002000000082540606001DA
:1002C000000102000105010902A10185020901A145
:1002D00000050919012908150025019508750181F6
:1002E000020501093009311581257F9502750881C4
:1002F0000609381581257F950175088106050C0AC8
:1003000038021581257F950175088106C0C0050159
:100310000980A101850319012AB700150126B7003C
:10032000950175108100C0050C0901A10185041912
:10033000012AA002150126A002950175108100C0B6
:1003400005010906A1018506050719E029E7150041
:1003500025019508750181020507190029EF15008F
:10036000250195F0750181020508190129059505FA
:1003700075019102950175039101C005010906A15E
:1003800001050719E029E715002501950875018188
:10039000029501750881010507190029FF1500263E
:1003A000FF009506750881000508190129059505C6
:1003B00075019102950175039101C00011241FBEC2
:1003C000CFEFDAE0DEBFCDBF11E0A0E0B1E0E4EFB7
:1003D000F5E402C005900D92A638B107D9F722E0E6
:1003E000A6E8B1E001C01D92AF38B207E1F70E9464
:1003F00071120C94F8220C940000559A209A0895DA
:1004000080FF02C05D9801C05D9A81FF02C02898FC
:100410000895289A089581E0089581E008950C9444
:100420000D0208950C9411021F93CF93DF9300D017
:1004300000D01F92CDB7DEB749835A836B833091CA
:10044000890189819A81311114C0662359F02223D0
:1004500049F00E94CD08182F682F89819A810E9447
:10046000740803C00E94A008182F69817A81812F27
:1004700004C00E94CD0869817A810F900F900F907F
:100480000F900F90DF91CF911F910C94F20FFC0110
:10049000262F408151816281738184810C941402E2
:1004A00081E00895CF93DF93EC0160E00E94470262
:1004B000BE01DF91CF910C9412020C9435110C9473
:1004C000311108950E941E070E9461022FEF84E3FC
:1004D0009CE0215080409040E1F700C000000C9467
:1004E0003D1B0F931F93CF93DF938C0161E00E941C
:1004F0004702EC01B8010E940F02882309F444C0AE
:10050000B801CE010E94F4158823F1F1B801CE01A3
:100510000E94DB188823C1F1B801CE010E94EF16BA
:10052000882391F1B801CE010E943718882361F128
:10053000F8018281882309F1CB358DE5D807C1F018
:1005400050F4C115FCE5DF0781F0CF3DDC45A9F48F
:100550000E94040E19C0CC35EDE5DE0761F0CD3503
:10056000DD4559F40E94470D08C00E9462020CC08C
:100570000E94500D02C00E94530DC801DF91CF911F
:100580001F910F910C940B0280E0DF91CF911F918E
:100590000F9108950E94721A80E00E9429160C940F
:1005A000E7020E9418150E94EA020C94781A0C9433
:1005B000000281E008950C94D9020895CF93C82FCA
:1005C0000E94D7028C2F0E94DB02CF91089580E019
:1005D0000C94DE020E9437190C94DE020E94371937
:1005E00090918801891721F0809388010C94DE0294
:1005F0000895CF93DF93CDB7DEB72B970FB6F8945E
:10060000DEBF0FBECDBF4F83588769877A878B8740
:1006100061110E94930C9E012F5F3F4F86E0F9010C
:1006200011928A95E9F785E0FE013796D90101908C
:100630000D928A95E1F789819A814C815D81452BE4
:1006400031F09F3F31F491E08F3F19F403C091E006
:1006500001C090E090FF09C049815A816B817C8183
:100660008D819E810E94B40B05C0C9010E94500279
:100670008111F2CF2B960FB6F894DEBF0FBECDBF1F
:10068000DF91CF910895FC01808191810E940F0933
:100690000895CF93882309F4A4C0C82F8238C1F4E9
:1006A0000E94371981FD9DC069E3809102019091FC
:1006B00003010E942D1A0E94B50C2FEF81EE94E0E9
:1006C000215080409040E1F700C0000069E319C06C
:1006D000833801F50E94371980FD83C063E580915E
:1006E0000201909103010E942D1A0E94B50C2FEF78
:1006F00081EE94E0215080409040E1F700C000007E
:1007000063E580910201909103010E94381ACF9114
:100710000C94B50C8438C1F40E94371982FD61C075
:1007200067E480910201909103010E942D1A0E94BA
:10073000B50C2FEF81EE94E0215080409040E1F71E
:1007400000C0000067E4DDCF8CEF8C0F813AD0F45D
:100750006C2F80910201909103010E94AD198823B2
:1007600049F06C2F80910201909103010E94381A88
:100770000E94B50C6C2F80910201909103010E94A0
:100780002D1AC5CF80E28C0F883048F4C77081E005
:1007900001C0880FCA95EAF70E94760CB8CFEBE546
:1007A000EC0FE33040F4F0E0E95BFE4F808190E035
:1007B000CF910C946B19E8E5EC0FE73150F4F0E0C1
:1007C000EE0FFF1FE75EFE4F80819181CF910C9469
:1007D0008119CD3E30F08C2F0E94F612CF910C94EF
:1007E000C813CF910895882309F464C0823879F43E
:1007F0000E94371981FF5EC069E3809102019091E8
:1008000003010E942D1A0E94B50C69E310C08338C1
:10081000B1F40E94371980FF4DC063E58091020159
:10082000909103010E942D1A0E94B50C63E58091FE
:100830000201909103010E94381A0C94B50C84387F
:1008400079F40E94371982FF35C067E48091020174
:10085000909103010E942D1A0E94B50C67E4E7CF26
:100860009CEF980F913A10F4682FE1CF90E2980F27
:10087000983050F4877091E001C0990F8A95EAF79B
:10088000892F0E947C0CD9CF9BE5980F933020F4E0
:1008900080E090E00C946B1998E5980F973120F464
:1008A00080E090E00C9481198D3E20F00E9451135D
:1008B0000C94C81308951F93CF93DF93182FEB0167
:1008C0000E944903209741F08FE99FE00197F1F7DB
:1008D00000C000002197F6CF812FDF91CF911F91AB
:1008E0000C94F303893319F060E070E002C060E516
:1008F00070E00C945B04882321F00E94760C0C9429
:10090000B50C0895882321F00E947C0C0C94B50C42
:100910000895CF92DF92EF92FF920F931F93CF93A0
:10092000DF937C01D62FC72FFC0112810581029530
:100930000F700E946C0C8823B9F01123A9F08C2F42
:10094000807F803421F080E28D0F883068F08091C4
:10095000720282FD09C082E00E94150D0E946C0C9B
:1009600091E0D82ED92601C0D12CCC2EC2948FE094
:10097000C8228C2D90E08C30910508F0CFC1FC018D
:10098000EA5AFF4F0C9489228C2F807FCF708823E6
:1009900011F0C295C07F112399F0CC2309F4AAC1AC
:1009A00080E28D0F883010F0D11104C08C2F0E948E
:1009B000760C03C08C2F0E94860C0E94B50C9AC145
:1009C0008D2F0E94F303CC2309F4A8C180E28D0F80
:1009D000883038F1DD2329F18C2F0E948C0C24C043
:1009E0008C2F807FCF70803211F0C295C07FDD23C5
:1009F00019F0D130A1F13DC08091720282FF17C081
:100A0000112349F0CC2329F08C2F0E94760C0E94F0
:100A1000B50C80E070C180E00E94F303CC2309F4A0
:100A20007DC18C2F0E947C0C0E94B50C77C11123D4
:100A300071F0002341F0013031F40E94960C8C2BB0
:100A40000E949E0C6BC10E94960C8C2B1DC0002333
:100A500019F0013009F462C10E94AB0C25C01123CA
:100A600021F0063008F05AC10EC0053008F056C11A
:100A70001BC0112361F0002331F0F701858180FF55
:100A800039C18F7085838C2F0E947B0447C100235E
:100A900059F0D93309F03FC1FFEF07EE13E0F150F1
:100AA00000401040E1F735C18C2F0E94820436C10E
:100AB0008C2F86958695837019F0813061F02EC158
:100AC000112321F08D2F9C2F937002C080E090E0C5
:100AD0000E946B192BC1112321F08D2F9C2F937035
:100AE00002C080E090E00E94811920C18D2F112367
:100AF00019F00E94F61202C00E9451130E94C813FE
:100B000015C18C2F837009F047C011110BC12D2F17
:100B1000229526952770220F220F6D2F6F70862F3A
:100B200090E0A0E0B0E0022E04C0880F991FAA1F39
:100B3000BB1F0A94D2F7D4FF10C04FE050E060E032
:100B400070E004C0440F551F661F771F2A95D2F727
:100B5000409550956095709503C040E050E0BA0113
:100B6000C695C695C3708A019B01082B192B2A2BA9
:100B70003B2BC901B801C23049F058F4C13019F01B
:100B80000E948A07CFC00E947807CCC00E949C07B1
:100B9000C9C00E947607C6C0112319F08C2F81703E
:100BA00001C08695882309F4BDC02D2F2295269576
:100BB0002770220F220F6D2F6F70862F90E0A0E01C
:100BC000B0E0022E04C0880F991FAA1FBB1F0A9411
:100BD000D2F7D4FF10C04FE050E060E070E004C0F6
:100BE000440F551F661F771F2A95D2F740955095E1
:100BF0006095709503C040E050E0BA01C695C69577
:100C0000C3708A019B01082B192B2A2B3B2BC9018E
:100C1000B801C23049F058F4C13019F00E944F08B1
:100C200081C00E943D087EC00E9461087BC00E9476
:100C3000B00778C0CF70112339F08C2F0E94D607EF
:100C40008D2F0E947B046EC08D2F0E9482048C2FFA
:100C50000E94F70767C0D23F21F128F4D03F41F04E
:100C6000D13FC1F043C0D33F19F1D43F79F03EC02A
:100C7000112341F0053008F051C08C2F8F710E9474
:100C80001C084CC0063008F049C0F7CF80917202B2
:100C900082FF18C0112339F08C2F8F710E94D60764
:100CA0003DC01123C9F38C2F8F710E94F70736C006
:100CB000112329F08C2F8F710E94C1072FC00E9431
:100CC000BC072CC0112349F0CF718C2F0E94D6078E
:100CD00063E08C2F0E94FA0C21C081E00E94150D68
:100CE0000230E0F082E00E94150D18C0112331F0AF
:100CF000002391F28D2F0E94490310C0002399F226
:100D0000D93349F41FEF27EE33E011502040304033
:100D1000E1F700C000008D2F0E94F30388EF8C0DD7
:100D2000843020F40E9437190E94DE02DD20C9F0D1
:100D30000E94680C80FD15C0F70112820E94620CAF
:100D40000E94D607C7010E94D2060E94620CDF9162
:100D5000CF911F910F91FF90EF90DF90CF900C9467
:100D6000F707DF91CF911F910F91FF90EF90DF90E8
:100D7000CF9008950F931F93CF93DF93EC01688179
:100D800079818A810E941A098C010E9473080E944D
:100D90006407B801CE010E948904DF91CF911F91B1
:100DA0000F910895CF93DF93EC01988189812B8176
:100DB0003C81232B31F08F3F31F481E09F3F19F4C8
:100DC00003C081E001C080E080FD1DC0CE010E9413
:100DD0007102811110C00E946C0C8823A1F08A81DD
:100DE000882389F08091720282FD0DC082E0DF913C
:100DF000CF910C94150DCE010E94BA06CE01DF9161
:100E0000CF910C945202DF91CF91089580E090E051
:100E10000E946B1980E090E00E9481190E94930C5F
:100E20000E94B50C0E94F9140C94C8138091020121
:100E3000909103010E94431A0C9406070E94830CB0
:100E40000C94160792959F70963079F010F492509A
:100E500001C09A50923068F4803F69F018F4883EDF
:100E600040F409C0843F29F406C0883E20F0813F49
:100E700011F080E0089581E00895FC018081918166
:100E80000E940F090E9422070895CF93DF9300D09C
:100E900000D01F92CDB7DEB70F900F900F900F903C
:100EA0000F90DF91CF910895CF93DF9300D000D0C2
:100EB00000D0CDB7DEB726960FB6F894DEBF0FBED2
:100EC000CDBFDF91CF910895089508950C946507E3
:100ED0000C9466070E9468076093A2017093A301B7
:100EE0008093A4019093A5010C9406070C946A07C3
:100EF0000F931F930091A2011091A3012091A401CF
:100F00003091A501602B712B822B932B1F910F9198
:100F10000C946A070F931F930091A2011091A301F3
:100F20002091A4013091A501602371238223932392
:100F30001F910F910C946A070F931F930091A201C8
:100F40001091A3012091A4013091A5016027712780
:100F5000822793271F910F910C946A070C946507C1
:100F60000E94AE0760939E0170939F018093A00141
:100F70009093A1010C94060760E070E0CB010C9403
:100F8000B0070F931F9341E050E060E070E08A01EA
:100F90009B0104C0000F111F221F331F8A95D2F737
:100FA000C901B8011F910F910C94B0070F931F93C3
:100FB00041E050E060E070E004C0440F551F661F40
:100FC000771F8A95D2F780919E0190919F01A09101
:100FD000A001B091A1018A019B01082B192B2A2B9A
:100FE0003B2BC901B8011F910F910C94B0070F93CF
:100FF0001F9341E050E060E070E004C0440F551FD3
:10100000661F771F8A95D2F7409550956095709529
:1010100080919E0190919F01A091A001B091A101AA
:101020008A019B01082319232A233B23C901B80104
:101030001F910F910C94B0070F931F9341E050E064
:1010400060E070E004C0440F551F661F771F8A954B
:10105000D2F780919E0190919F01A091A001B09143
:10106000A1018A019B01082719272A273B27C901CB
:10107000B8011F910F910C94B0070F931F9300912B
:101080009E0110919F012091A0013091A101602B40
:10109000712B822B932B1F910F910C94B0070F9300
:1010A0001F9300919E0110919F012091A00130910A
:1010B000A10160237123822393231F910F910C942C
:1010C000B0070F931F9300919E0110919F012091F3
:1010D000A0013091A10160277127822793271F91DA
:1010E0000F910C94B0070895292F220F920F990F9A
:1010F000890FE82FE695E695E695877051E001C0E7
:10110000550F8A95EAF785E0E89FF0011124E6572C
:10111000FE4F20E030E070E04081CB01022E02C0A3
:10112000969587950A94E2F78170819584278523A7
:10113000842781932F5F3F4F2530310569F708954C
:10114000292F220F920F990F890F682F66956695A8
:101150006695982F977085E0689FB001112440E054
:1011600050E080E0FB01E40FF51FE657FE4F2081C1
:1011700030E0092E02C0369527950A94E2F72170D7
:101180003327042E01C0220F0A94EAF7822B4F5F07
:101190005F4F4530510531F70895BF92CF92DF92EE
:1011A000EF92FF920F931F93CF93DF938C01C09028
:1011B0009E01D0909F01E090A001F090A10180914C
:1011C000A2019091A301A091A401B091A501C82A08
:1011D000D92AEA2AFB2ACFE1D0E0D701C6010C2E9A
:1011E00004C0B695A795979587950A94D2F780FD88
:1011F00004C0219790F7B12C07C0BC2EB8018C2FEA
:101200000E9405100197A9F38B2DDF91CF911F91BB
:101210000F91FF90EF90DF90CF90BF900895CF9304
:10122000DF93EC010E94CD08BE010E940510DF9102
:10123000CF9108951F93CF93DF93EB019091890194
:10124000992321F0CB010E940F0913C0882349F094
:10125000CB010E94CD08182F682FCE010E94740880
:1012600004C0CB010E94A008182FBE01812F0E944C
:101270000510DF91CF911F9108951F93CF93DF93B6
:10128000C091A60116E08091A701C81799F0D0E09F
:101290001C9FF0011D9FF00D1124E855FE4F408169
:1012A000518162817381848195810E9454072196C6
:1012B000C770E9CFDF91CF911F9108954091D80178
:1012C0005091D9016091DA017091DB018091DC01CC
:1012D0009091DD010C945407EF92FF920F931F93AE
:1012E000CF93DF938091DD0182958F7009F065C007
:1012F0008091DA01882309F460C08091A601F09002
:10130000A7011091D8010091D9016091DB01709182
:10131000DC0191E01F3F09F090E0C0910001D09105
:101320000101292F96E0E92E8F1509F446C06115B9
:10133000710521F00F3F21F030E003C031E001C022
:10134000322F90E030FD36C0E89EF001E99EF00DAE
:101350001124DF01A855BE4F11963C91119730130F
:1013600029C03C91311326C012963C91129731113D
:1013700021C013964D915C911497461B570B4C1747
:101380005D07C0F48091DD018F7080618093DD0185
:10139000E355FE4F80818F708061808388ED91E0FE
:1013A0000E94D206DF91CF911F910F91FF90EF9095
:1013B0000C943D0901968770B7CFDF91CF911F91B3
:1013C0000F91FF90EF9008959F92AF92BF92CF92AE
:1013D000DF92EF92FF920F931F93CF93DF93CDB7DE
:1013E000DEB761970FB6F894DEBF0FBECDBF8C019C
:1013F00085E0F801DE011D9601900D928A95E1F7D6
:10140000D8011296EC909091D801E091D9012091E9
:10141000DB013091DC012115310531F0EF3F31F472
:1014200081E09F3F19F403C081E001C080E0B82F44
:10143000B1709B2E80FD47C1D8014C9111965C91F3
:1014400011971396AD90BC90149788EDC82E81E04B
:10145000D82EF090DA01B501621B730B20910001C8
:1014600030910101FF2009F4D9C08091DD0162179C
:10147000730708F095C0282F207F09F052C05E1333
:1014800013C0491311C0FE2CE1100EC08F70806193
:101490008093DD010E945E09C6010E94D206809100
:1014A000DD01F80185834DC1AB2831F05F3F31F498
:1014B00081E04F3F19F403C081E001C080E080FD6E
:1014C00003C081E08E2502C080E090E0F82FF1702B
:1014D000FF2E80FF1CC08091A6012091A70136E05D
:1014E000821709F40BC190E0389FF001399FF00D8D
:1014F0001124E855FE4F6181561306C060814613E2
:1015000003C06281E61203C001968770E9CFFE2C0A
:10151000EE2009F416C18091DD0181608093DD0128
:1015200054C05E1306C0491304C0E11002C0F801A4
:1015300099C0C8010E943D07882361F1EE2051F156
:101540002091DD01822F82958F7090E0029774F0D8
:101550008091D8019091D90198878F831986BB8695
:10156000AA862C87CE0107960E94D20686E0F80153
:10157000A8EDB1E001900D928A95E1F70E946C0907
:101580000E945E090AC05E1711F1C8010E943D0762
:1015900081112CC0C8010E94D206FF24F394D1C04F
:1015A000282F207F81F77A2DB98AA88A6E2D898904
:1015B0000E94450788ED91E00E94D20686E0D601A0
:1015C0001D928A95E9F70E945E09F12CBAC0491371
:1015D000DCCFE110DACFF8018583C8010E94D20682
:1015E00086E0D6011D928A95E9F7ABC0EE2091F214
:1015F0002091DD01822F82958F7090E002970CF48C
:10160000B5CF8091D8019091D9019A8389831B82AB
:10161000BD82AC822E83CE010196A6CF62177307DE
:1016200008F044C0FE2CEE2009F4B4CF5E1330C0A5
:1016300049132EC02091DD0120FD21C0822F82950B
:101640008F70482F50E041155105C9F0F8012583EE
:101650004F30510541F08F5F982F9295907F822FE8
:101660008F70892B8583C8010E94D20686E0F8011D
:10167000A8EDB1E001900D928A95E1F73CC086E0BB
:10168000F801A8EDB1E001900D928A95E1F759C0FB
:10169000C8010E943D07811169CF8091DD01816001
:1016A0008093DD01C8010E94D2064BC07A2DB98A11
:1016B000A88A6E2D89890E94450786E0D6011D9271
:1016C0008A95E9F718C0EE2009F464CFC8010E949A
:1016D0003D07F82E882309F45DCF86E0F801A8EDD8
:1016E000B1E001900D928A95E1F788ED91E00E94BA
:1016F00043030E946C090E945E0923C04D875E87E8
:101700008D859E850E940F09292F22952F702230EA
:1017100028F49F7039F0811105C00BC0243028F4E3
:101720009F7049F4805E883020F0C8010E94D20684
:101730009F2CF92C06C0D80115969C91907F91F7AB
:10174000F8CF8F2D61960FB6F894DEBF0FBECDBFD8
:10175000DF91CF911F910F91FF90EF90DF90CF908D
:10176000BF90AF909F9008951F93CF93DF93CDB715
:10177000DEB72C970FB6F894DEBF0FBECDBF4F83F8
:10178000588769877A878B879C87CE0107960E9446
:10179000E4098823D1F09F8188852A853B85232B06
:1017A00031F08F3F31F481E09F3F19F403C081E0B5
:1017B00001C080E080FD47C04F81588569857A85EA
:1017C0008B859C850E9454073EC086E0FE013796BB
:1017D000DE01119601900D928A95E1F7FF81E8856F
:1017E0006A857B856115710531F0EF3F31F481E049
:1017F000FF3F19F403C081E001C080E080FD23C0F9
:101800002091A70130E0C901019687709927409186
:10181000A60150E084179507F1F1F983EA837D83EF
:101820006C8396E0929FD001939FB00D1124A85530
:10183000BE4FFE01319601900D929A95E1F780938B
:10184000A7010E943D0916E08091A6019091A70191
:10185000891771F1189FC001112488559E4F0E946D
:10186000E409882329F1E091A6011E9FF0011124CB
:10187000E855FE4F40815181628173818481958159
:101880000E9454078091A60190E0019687709927E5
:101890008093A601D9CF0E941E071092A701109233
:1018A000A601E8EDF1E086E0DF011D928A95E9F7F7
:1018B0002C960FB6F894DEBF0FBECDBFDF91CF914F
:1018C0001F9108958091FE018595859585950895D0
:1018D0008091FE01877008959091FE01977081E0DC
:1018E00009F480E0089580912102089590912102E9
:1018F000892B80932102089580959091210289235C
:10190000809321020895109221020895909120025F
:10191000892B80932002089580959091200289233D
:101920008093200208951092200208958091FF0173
:10193000089508950C94990C0C949A0C909172024D
:1019400092FD08C09091FF01981721F08093FF014C
:101950000C949C0C08958091FF01882329F010922B
:10196000FF0180E00C949C0C0895CF93DF93E091ED
:101970000201F0910301809121028083E091020134
:10198000F0910301908180912002892B80838091C6
:10199000FF01882381F0E0910201F0910301908121
:1019A000892B808380910201909103010E949719F5
:1019B00081110E94AB0CC0910201D091030140E261
:1019C00050E06EED71E0CE010E94A922892B69F0F2
:1019D00080E2FE01AEEDB1E001900D928A95E1F753
:1019E000CE01DF91CF910C944319DF91CF910895EF
:1019F0000C94990C9091720292FD10C098E0899F0E
:101A000090011124262B2093FE010E94D60780917D
:101A1000FE018595859585950C94F80C0C94D60758
:101A20001092FE0180E00C94F80C2091FE0180954C
:101A300082238093FE01982F977099F430E0482F0D
:101A4000082E000C550B2417350759F0909172029F
:101A500092FD07C08595859585950E94F7070C94A2
:101A6000100D08959091720292FB222720F92817F9
:101A700069F080FB92F990937202809171029091CB
:101A800072020E94800D82E00C94150D08958091E1
:101A9000720282FB882780F991E089270C94320D2D
:101AA00081E00C94320D80E00C94320D6FEF7FEFEB
:101AB00080E090E00C94E22280E090E00E94BE2260
:101AC00021E0893E9E4F09F020E0822F089582E0B8
:101AD00090E00C94B62283E090E00C94B622CF9371
:101AE00084E090E00E94B622C82F82E290E00E943B
:101AF000B6222C2F30E0A901582BCA01CF910895AE
:101B0000CF93C92F682F84E090E00E94C4226C2FED
:101B100082E290E0CF910C94C422AB01BC018FE033
:101B200090E00C94D622AB01BC0183E190E00C94D0
:101B3000D62260E070E0CB010C94930D60E070E081
:101B4000CB010E948D0D0C94990D69EE7EEF80E023
:101B500090E00E94E22260E082E090E00E94C422D5
:101B600060E083E090E00E94C4221092A2011092F3
:101B7000A3011092A4011092A50160E084E090E01E
:101B80000E94C42260E082E290E00E94C42260E0F1
:101B900085E090E00E94C42260E086E090E00E9430
:101BA000C4226FEF87E090E00E94C42240E050E042
:101BB000BA0188E090E00E94D62260E08DE090E0DB
:101BC0000E94C42240E050E0BA0188E190E00E9407
:101BD000D62260E087E190E00E94C42240E050E01D
:101BE000BA018CE190E00E94D62260E070E080E2D1
:101BF00090E00E94E22240E050E0BA0188E190E0EB
:101C00000E94D6220C949E0D0C94A50D682F8EE098
:101C100090E00C94C4220E94FC1A60932B027093F3
:101C20002C0280932D0290932E02609327027093D2
:101C300028028093290290932A02089585B780682C
:101C400085BF85B7806885BF089581E008950C94AD
:101C5000250E08950C94290E0C94290E0C942C0E2C
:101C60000C94FD010C94290E0E941E0E81EE90E151
:101C70000E942D190E94320E0C94300E0E942A0EE2
:101C80000C94290E0E94FB100E94DD020C94DF16BA
:101C90000E94E71A0E94D2110E94420E0E9418155B
:101CA0000C942E0E8F929F92AF92BF92CF92DF92A2
:101CB000EF92FF920F931F93CF93DF93CDB7DEB7D1
:101CC0002A970FB6F894DEBF0FBECDBF0E94E71172
:101CD000982E81110E940B0E82E2A82E82E0B82E6F
:101CE00000E010E0802E802F0E941F11D82EF501F9
:101CF000C1905F01C826B1F40F5F1F4F0530110579
:101D000089F78FEF89838A831B820E94F01A816092
:101D1000782F9D838C8349815A816B818D810E94AC
:101D2000F9022FC080912F0281FD0E942511E12C24
:101D3000FF24F3948C2D8F21F1F00E94270E88232D
:101D400099F0EE828F82DF2081E009F480E08887BD
:101D50000E94F01A8160782F9A8789874E815F816F
:101D600068858A850E94F902F801EE5DFD4F808149
:101D7000F826F08206C0E394FF0CF6E0EF12DACF0B
:101D8000BBCF81E0911001C080E02A960FB6F89495
:101D9000DEBF0FBECDBFDF91CF911F910F91FF909E
:101DA000EF90DF90CF90BF90AF909F908F9008956D
:101DB0000E94520E0E94DE160E94E6130C94EE0260
:101DC000CF93DF930E940A10EC01811521E5920761
:101DD00008F045C0811530E5930708F094C0883EAF
:101DE000910528F5803E910508F0F8C0883A9105E4
:101DF00070F4853A910508F07CC08130910509F4B2
:101E000075C008F4E8C0049708F0E8C0E4C08F3B50
:101E1000910508F0E0C0C85AD0E0CC0FDD1FC65BCA
:101E2000DE4F0990D881C02DCE019464D8C08115B1
:101E300040E2940758F4811551E0950708F0CEC0B0
:101E40008D3E910508F4C7C09065C9C0C11580E4F6
:101E5000D80708F4C0C0DF70CE01906AC0C08115F9
:101E600025E59207A8F4811534E5930708F095C09D
:101E7000811543E5940708F07BC0811552E595076D
:101E800008F061C0D82FCC27CE01816F906AA7C01F
:101E9000C11589E5D807A0F4C11528E5D20708F0D7
:101EA00082C0C11536E5D30708F095C08C2F0E947B
:101EB0009E108F7190E0D82FCC27CE0190628FC0FA
:101EC000C1154AE5D40708F474C0CE0190568115B7
:101ED000904208F080C08D2F8F710E949E10DD27E8
:101EE000D0628F71AE01582BCA0179C081E090E0B9
:101EF00076C0C55AD0E0C858DE4F8881C82FD0E0E0
:101F0000CE0190646CC074E0969587957A95E1F760
:101F1000282F23703C2F337081E090E002C0880F9F
:101F2000991F3A95E2F79C68AC01522B9A019C2FBD
:101F30009F709695969550E2959FE0011124C901F6
:101F40008C2B9D2B4CC08370992721E030E002C080
:101F5000220F331F8A95E2F79C2F9695969580E283
:101F6000989FE0011124C22BD32BCE019C6837C06F
:101F70008370992721E030E002C0220F331F8A9539
:101F8000E2F79C2F9695969540E2949FE0011124EC
:101F9000C22BD32BCE019A6822C0D82FCC27CE01DA
:101FA000846F906A1CC0DC2FCC27CE01806F906AB2
:101FB00016C08C2F8F700E949E1094E0D695C79506
:101FC0009A95E1F7CF70D0E0DC2FCC27D0699E0145
:101FD000282BC90104C080E090E001C0CE01DF9150
:101FE000CF9108952EE1829FC0011124FC0126E0CB
:101FF000729FE00DF11D1124E60FF11DEE0FFF1F82
:10200000E852FF4F8591949108950E94F20F0E942B
:10201000E00E08958238910569F1B0F4813391059D
:1020200009F46DC048F48932910509F463C08A321D
:10203000910509F469C008958533910509F455C0E7
:1020400089339105B9F00895833E910569F138F41B
:10205000803E9105B1F0823E910509F10895863EDA
:102060009105A9F1873E9105B9F1843E910509F0EA
:1020700064C023C02091710220FD4FC021FD4DC0DE
:1020800008958091710280FD44C08091720280FFAA
:1020900044C08091710284FD42C083EE4DC08091A6
:1020A000710282FF38C0F5CF8091710282FD33C08A
:1020B0008091720280FD31C0ECCF8091720281FF6D
:1020C00032C08091710284FD2AC087EE35C08091B4
:1020D000710283FF26C0F5CF8091710283FD21C07C
:1020E0008091720281FD1FC0ECCF8091710285FD4D
:1020F0001CC01DC08091710285FD19C016C0809161
:10210000710286FD16C017C08091710286FD13C052
:1021100010C089E311C082EE0FC080EE0DC080E0D8
:102120000BC086EE09C084EE07C089E205C085E3D6
:1021300003C08AE201C081E390E0089590917102AA
:1021400092FF0DC0282F2871283019F4877F8460F2
:1021500006C0282F2471243011F48B7F886093FFF0
:102160000DC0282F2871283119F4877E846106C09C
:10217000282F2471243111F48B7E88612091720202
:1021800020FF0DC0382F3871383019F4877F8160F7
:1021900006C0382F3171313011F48E7F886021FFF5
:1021A0000DC0282F2871283119F4877E816106C05F
:1021B000282F2171213111F48E7E886194FD877E54
:1021C000089580E008950C94560D0E94E7118FE366
:1021D0009CE90197F1F700C000000E94E71180E040
:1021E0000E941F1180FF04C00E94E3100C943D1B4D
:1021F00008950C94E5100E945C0D811102C00E94AC
:10220000040E0E94670D80932F020E946F0D909321
:102210007202809371020E94F9100E946B0D682F68
:1022200070E080E090E00E94760760919E017091DE
:102230009F018091A0019091A1010C94AE07E82F1D
:10224000F0E0E858FD4F80810895089580EA8A956E
:10225000F1F7089500C008950C94261108950C9488
:102260002E110C942F110C942E110C943311F89400
:10227000E82FE295EF70F0E031A1282F2F7081E078
:1022800090E001C0880F2A95EAF7982F9095932344
:1022900091A392A1892B82A3789408950F931F9301
:1022A000CF93DF93C1E8D1E089918F3F11F00E9475
:1022B000371181E0C638D807B9F7CBE7D1E001E89C
:1022C00011E089918F3F11F00E9437110C171D0703
:1022D000C1F7DF91CF911F910F910895CF92DF92B7
:1022E000EF92FF920F931F93CF93DF938C01C62F32
:1022F000D0E0CE018F579E4F7C01FC0190819F3F23
:1023000009F447C0D62EF894E92FE295EF70F0E07B
:1023100081A19F7021E030E001C0220F9A95EAF779
:10232000822B81A382A12095282322A378940E9446
:102330002A11EBE7F1E041E851E031E0C12C2191B5
:102340002F3F89F0A22FA295AF70B0E090968C91AC
:1023500090E02F7002C0959587952A95E2F780FD51
:1023600002C0832F01C080E0C82A330F4E175F07D9
:1023700031F7F70180818F3F11F00E94371161E042
:10238000C11001C060E08D2D0E942C11C00FD11F23
:10239000C882DF91CF911F910F91FF90EF90DF9056
:1023A000CF9008950E944E1185E0E8E7F2E0DF014A
:1023B000982F1D929A95E9F7E3E7F2E0DF011D926D
:1023C0008A95E9F785E00E942E120C945D02FF9237
:1023D0000F931F93CF93DF9300D000D01F92CDB700
:1023E000DEB78E010F5F1F4F85E0F80111928A95CD
:1023F000E9F7F12C6F2DC8010E946E11F394F5E0FE
:10240000FF12F8CF45E050E0B80183E792E00E9468
:10241000A922FF24F394009709F4F12C892B41F0B1
:1024200085E0F801A3E7B2E001900D928A95E1F70B
:102430002F2D45E068E772E083E792E00E942F12BB
:102440000E945F028F2D0F900F900F900F900F90B2
:10245000DF91CF911F910F91FF9008950895FF9202
:102460000F931F93CF93DF938C01F62ED72FC42F9A
:10247000222349F081E0809332020E94F01A909367
:10248000310280933002809132028823C1F0809122
:102490003002909131020E94081B059780F0EF2DC9
:1024A000FD2FD8014C2F50E0CD01801B910B8417DC
:1024B00095071CF48D918193F7CF10923202DF9132
:1024C000CF911F910F91FF9008950E94F51C0E94DB
:1024D000480E0C94011D0E94051D0E94D80E0C94FC
:1024E0001F1D0E948E1A0E94DC1C0E94340E0E9446
:1024F00065120E946B120E943E0EFBCF8091390242
:1025000080FF06C06091090170E0660F771F26C04A
:1025100081FF04C06091090184E005C082FF07C00B
:102520006091090188E0689FB001112417C0909163
:1025300038029923D1F060910801961788F720910D
:10254000090188E0289F90011124929FA001939F88
:10255000500D112470E0CA010E94532260387105A9
:1025600040F46115710519F406C068E070E0862F2B
:1025700008958FE7089581E008958091390280FFE2
:1025800008C06091050170E0759567957595679530
:1025900021C081FF06C06091050170E075956795C7
:1025A00019C082FF04C06091050170E010C09091D5
:1025B0003702992399F0609104019617A0F7809152
:1025C0000501899FC001112470E00E9453226038E8
:1025D000710540F46115710519F406C061E070E001
:1025E000862F08958FE7089581E008958D3E21F4A8
:1025F0000E947E12819504C08E3E29F40E947E12B4
:1026000080933D0208958F3E21F40E947E128195B1
:1026100004C0803F29F40E947E1280933C020895FA
:10262000893F19F40E94BD1205C08A3F31F40E940F
:10263000BD12819580933E0208958B3F21F40E9444
:10264000BD12819504C08C3F29F40E94BD12809375
:102650003F0208959FE0980F983078F421E030E031
:10266000A90102C0440F551F9A95E2F7CA01909143
:102670003B02892B80933B0208958D3F21F480918A
:10268000390281600BC08E3F21F480913902826053
:1026900005C08F3F29F4809139028460809339020C
:1026A00008958D3E39F490913D0297FF35C0109208
:1026B0003D0259C08E3E29F490913D021916BCF39B
:1026C0002BC090913C028F3E29F497FF25C01092B9
:1026D0003C0249C0803F19F41916CCF31DC09091FB
:1026E0003E02893F29F41916BCF410923E023BC009
:1026F0008A3F19F497FF10C0F8CF8B3F39F49091BF
:102700003F0297FF09C010923F022DC08C3F21F479
:1027100090913F021916BCF39FE0980F983080F417
:1027200021E030E0A90102C0440F551F9A95E2F75D
:10273000CA01809590913B02892380933B0213C08C
:102740008D3F21F4809139028E7F0BC08E3F21F4A2
:10275000809139028D7F05C08F3F29F48091390225
:102760008B7F8093390280913C02811106C0809159
:102770003D02811102C01092380280913E02811107
:1027800006C080913F02811102C010923702089565
:102790000E94F01A20913C02211104C020913D02B8
:1027A000222321F0909336028093350220913E023D
:1027B000211104C020913F02222321F09093340282
:1027C000809333028AE392E00C945D19EF92FF92BA
:1027D0000F931F93CF93DF9300D000D000D0CDB7DD
:1027E000DEB786E0EAE3F2E0DE01119601900D9299
:1027F0008A95E1F7E0903C02F0903D0200913E02A4
:1028000010913F0210923C0210923D0210923E0243
:1028100010923F02E11003C0FF2009F45DC08091D7
:102820003502909136020E94081BAC01909138024B
:10283000992339F020910A0130E02417350758F028
:102840004BC020910B018AE0289F9001112424178E
:10285000350718F041C09F3F19F09F5F90933802F1
:10286000EE2061F00E947E121E1414F09FEF01C052
:1028700091E0989F902D112490933C02FF2061F0ED
:102880000E947E121F1414F09FEF01C091E0989FE8
:10289000902D112490933D0230913C023323E1F0BE
:1028A00020913D022223C1F045EB3403C0011124E5
:1028B000992319F090933C0203C081E080933C027D
:1028C00035EB2303C0011124992319F090933D02A5
:1028D00003C081E080933D02011103C0112309F47C
:1028E0005DC080913302909134020E94081BAC01BC
:1028F00090913702992339F02091060130E0241796
:10290000350758F04BC0209107018AE0289F9001BD
:1029100011242417350718F041C09F3F19F09F5F1D
:1029200090933702002361F00E94BD12101614F03C
:102930009FEF01C091E0989F902D112490933E024B
:10294000112361F00E94BD12111614F09FEF01C017
:1029500091E0989F902D112490933F0230913E0278
:102960003323E1F020913F022223C1F045EB3403F1
:10297000C0011124992319F090933E0203C081E015
:1029800080933E0235EB2303C0011124992319F0F3
:1029900090933F0203C081E080933F0280913C020C
:1029A00081110BC080913D02811107C080913E02D0
:1029B000811103C080913F0281110E94C813EB82F4
:1029C000FC820D831E8386E0FE013196AAE3B2E00D
:1029D00001900D928A95E1F726960FB6F894DEBF26
:1029E0000FBECDBFDF91CF911F910F91FF90EF9060
:1029F0000895EAE3F2E086E0DF011D928A95E9F7A7
:102A0000109238021092370210923902089586E02F
:102A100090E00C94B622682F86E090E00C94C422DB
:102A200080917D028470896180937D020C940B15E6
:102A30000E945C0D811104C00E94040E0E941015BA
:102A40000E94071580937D02282F269526952695AE
:102A500030E02430310524F08770886180937D0256
:102A600080917D0280FF04C086958695869501C081
:102A700080E00C94291620917D02822F8695869500
:102A80008695482F50E04330510554F48F5F982FBE
:102A9000990F990F990F822F8770892B80937D0250
:102AA00080917D02816080937D020E940B15809150
:102AB0007D028695869586950C94291680917D02D7
:102AC000982F969596959695A1F0915E990F990FEE
:102AD000990F8770892B80937D02887F91E009F49C
:102AE00090E080917D0290FB80F980937D020E94AE
:102AF0000B1580917D028695869586950C942916F6
:102B000080917D0280FD13C0816080937D028130C1
:102B100019F489E080937D0280917D020E940B155B
:102B200080917D028695869586950C942916089548
:102B300080917D0280FF08C08E7F80937D020E947D
:102B40000B1580E00C942916089580917D0280FD7C
:102B50000C9498150C94801590917D02892F869580
:102B6000869586958F5F8F719770843038F4880FC3
:102B7000880F880F892B80937D0202C090937D027D
:102B800080917D02887F91E009F490E080917D0240
:102B900090FB80F980937D020E940B1580917D024D
:102BA0008695869586950C942916843008F083E0E6
:102BB00090917D029770282F220F220F220F922BC7
:102BC00090937D02987F21E009F420E090917D02AE
:102BD00020FB90F990937D020C9429160E94D51544
:102BE00080917D020C940B159C01FB01828188234E
:102BF00049F12E3BFCE53F07C9F040F42C3BECE5E6
:102C00003E0769F02D3B3C4561F00895203C9CE572
:102C1000390791F070F0213C3C4589F0089583E03C
:102C200001C080E00E94EE1580E008950E945E15CC
:102C3000FBCF0E943B15F8CF0E94A515F5CF0E944F
:102C4000AC15F2CF81E00895259A2D9808952D981E
:102C500008958F929F92AF92BF92CF92DF92EF92A0
:102C6000FF920F931F93CF93DF93C82F843050F4BC
:102C7000811109C0809180008F77809380000E942D
:102C8000271606C0C3E08091800080688093800092
:102C9000A0918600B09187002C2F30E00E948F22F7
:102CA00023E030E040E050E00E9467220027122F2E
:102CB000232F342F012F122F232F332780918600AB
:102CC000909187006CE070E00E943F2260177107CE
:102CD00030F0C80169E070E00E943F225EC0809140
:102CE000860090918700E0908600F0908700E09148
:102CF0008600F0918700C6E0D0E0BE010E943F222E
:102D0000060F171F211D311D4801590185E0880C50
:102D1000991CAA1CBB1C8A95D1F7C701BE010E9451
:102D20003F226F01E12CF12CA7019601260F371FDE
:102D3000411D511DC501B4010E94672269017A013C
:102D4000E0918600F0918700CA01B9010E942F220C
:102D50009B01AC01DF010E949E229B01AC01C701D7
:102D6000B6010E942F22DC01CB012FE0B695A7957A
:102D7000979587952A95D1F7009186001091870045
:102D800020E030E0081719072A073B0728F4609174
:102D9000860070918700CB01BC017093890060931D
:102DA0008800DF91CF911F910F91FF90EF90DF90FE
:102DB000CF90BF90AF909F908F90089508950E94FC
:102DC000241682E88093800089E1809381008FEF50
:102DD0009FEF90938700809386000C941815CF93F3
:102DE000DF93EC01FB018281882309F43CC1C430EC
:102DF000FDE5DF0760F4CB3F9CE5D90788F49E0131
:102E000022503C452431310508F02EC109C0C2369C
:102E1000EDE5DE0729F0C63AFDE5DF0709F024C13C
:102E20000E946F0D9093720280937102C1318CE504
:102E3000D80709F4C6C008F042C0C930ECE5DE0787
:102E400009F49BC000F5C5308CE5D80709F485C0AE
:102E500078F4C330ECE5DE0709F478C008F07AC0F6
:102E6000C230DC4509F0F5C0809171028160EFC08D
:102E7000C7309CE5D90709F478C008F07AC0809182
:102E800071028061E4C0CD30FCE5DF0709F487C042
:102E900058F4CB309CE5D90709F479C008F07BC021
:102EA0008091710288606FC0CF30FCE5DF0709F4C4
:102EB00080C008F082C080917102877FC8C0CE3F79
:102EC0009CE5D90709F471C000F5C531FCE5DF07C1
:102ED00009F485C068F4C3319CE5D90709F475C0CD
:102EE00008F095C00E941E07809171028F77AFC0D5
:102EF000CC3FFCE5DF07A9F108F054C0CB3FDC452F
:102F000009F0A7C08091720240C0C230EDE5DE0733
:102F100009F489C058F4C1158DE5D80709F45AC0E1
:102F200008F069C08091720282602FC0C236EDE560
:102F3000DE0709F47CC0C63AFDE5DF0709F481C06D
:102F4000C330DD4509F085C080E06EC0809171021C
:102F500082607DC08091710216C08091710288608C
:102F600076C08091720282604FC08091710280624F
:102F70006EC08091710280646AC00E941E078091B9
:102F80007102806864C0846062C081603DC08091CD
:102F900071028E7F5CC0809171028D7F58C08091DC
:102FA000710216C08091720218C0809172028D7FEA
:102FB0002BC0809171028F7E4AC0809171028F7DFB
:102FC00046C0809171028F7B42C080917102877FE1
:102FD0008B7F3DC0809172028D7F8E7F15C0809166
:102FE000710282FB222720F991E0922790FB82F95F
:102FF00090FB83F92CC080917202982F909591706C
:103000008E7F892B90FB81F98093720222C00E94EF
:103010001E078091710287FB222720F991E09227F9
:1030200090FB87F914C081E00E94060E12C08091C7
:10303000710284FB222720F991E0922790FB84F90A
:1030400006C080917102982F909590FB80F9809333
:10305000710280917102909172020E94800D0E9413
:103060001E0780E001C081E0DF91CF910895CF93EA
:10307000DF9386319C4541F5EB010E94730C982F3C
:103080008A812091020130910301882379F09A7A94
:1030900081E009F480E080934002911102C069E26E
:1030A00001C065E3C9010E942D1A0AC08091400247
:1030B000811102C069E201C065E3C9010E94381AAA
:1030C0000E94B50C80E001C081E0DF91CF910895AE
:1030D0000F931F93CF93DF93C42FD22FFC018281D4
:1030E0008823C9F0409343020E94F01A9093420251
:1030F0008093410280E28C0F883008F057C0C7707F
:1031000081E001C0880FCA95EAF7DF91CF911F9146
:103110000F910C947B0480914302481330C080913E
:103120004102909142020E94081B883C910538F5AB
:1031300010E21D0FCD17B9F080E28C0F883040F4FB
:10314000C77081E001C0880FCA95EAF70E94820427
:10315000183028F581E09D2F977001C0880F9A954F
:10316000EAF70E947B04802F0E9472041830F0F46A
:10317000D77081E001C0880FDA95EAF70AC080E2D3
:103180008C0F883098F4C77081E001C0880FCA9511
:10319000EAF7DF91CF911F910F910C948204802F59
:1031A000DF91CF911F910F910C947204DF91CF9119
:1031B0001F910F9108950F939C01CB01243F4CE583
:1031C000340731F188F4293DFCE53F07D9F02A3D69
:1031D0004CE5340779F1283D3C45A9F506E221EE9E
:1031E00041EE68ED7CE52BC0263FFCE53F07E1F0B2
:1031F000A8F0273F3C4539F507E225EE46EE67EF9C
:103200007CE51DC007E225EE45EE69ED7CE517C0C3
:1032100006E221EE40EE64EF7CE511C007E225EE08
:1032200044EE65EF7CE50BC006E221EE42EE66EF70
:103230007CE505C008E221E045EE6AED7CE50E94F0
:10324000681880E008C0FC018281882319F0109280
:10325000430201C081E00F9108959093870180930C
:103260008601089590934902809348020895E09161
:103270004802F0914902309721F00190F081E02D51
:10328000099480E00895E0914802F0914902309756
:1032900099F020911801222359F02091710227FF03
:1032A00007C0DC012C9111962C93119726E02C93EA
:1032B0000280F381E02D09940895E0914802F09195
:1032C0004902309739F022E0DC012C930480F5812B
:1032D000E02D099408952091460230914702281765
:1032E000390771F09093470280934602E0914802BB
:1032F000F0914902309721F00680F781E02D099482
:10330000089520914402309145022817390771F041
:103310009093450280934402E0914802F091490263
:10332000309721F00084F185E02D09940895FC0187
:10333000329680911801882331F08091710287FFC5
:1033400002C09EE101C096E080E0915028F02191FA
:103350002223D9F38F5FF9CF0895662351F120918D
:1033600018012223E9F02091710227FF19C0462F8E
:103370004695469546954E31E0F4677021E030E081
:1033800002C0220F331F6A95E2F7FC01E40FF11D22
:10339000828190E02823392381E0232B69F409C03E
:1033A000FC01329608962191621729F0E817F90777
:1033B000D1F780E0089581E008959C01FC013296E8
:1033C0009FEF80E04191461789F09F3F19F441112A
:1033D00001C0982F8F5F8630A9F79F3F39F0F90120
:1033E000E90FF11D97FDFA956283089508959C01F8
:1033F0002A5F3F4FFC014281461301C012820196B1
:1034000082179307B9F70895262F269526952695B6
:103410002E3168F4FC01E20FF11D677021E030E00D
:1034200001C0220F6A95EAF78281282B2283089532
:10343000262F2695269526952E3170F4FC01E20F55
:10344000F11D677021E030E001C0220F6A95EAF7B4
:103450002095828128232283089520911801222318
:1034600029F02091710227FD0C94041A0C94DD19A7
:1034700020911801222329F02091710227FD0C943C
:10348000181A0C94F71920911801FC013296222386
:1034900031F08091710287FF02C08EE101C086E0A9
:1034A000DF011D928A95E9F7089508950C94551A45
:1034B00083E080934A020C94561A811102C081E085
:1034C00001C082E080934A020C94561A0C945D1A53
:1034D00081E080934A020C94561A0C94681A08955D
:1034E0000C946F1A0C94701A0C946F1A0C946F1A37
:1034F0000C946F1ACF930E94761A0E94E7110E94D3
:10350000741AC0E08C2F0E941F11811104C0CF5F7C
:10351000C530C1F701C081E0CF91089508951F9291
:103520000F920FB60F9211248F939F93AF93BF9377
:1035300080914B02811113C080917E0290917F0295
:10354000A0918002B09181024196A11DB11D80938E
:103550007E0290937F02A0938002B0938102BF917C
:10356000AF919F918F910F900FBE0F901F90189564
:1035700080918602843031F10E94CA0210924B027F
:1035800020E488E190E00FB6F894A895809360005D
:103590000FBE2093600083B7817F846083BF83B7B1
:1035A000816083BF7894889583B78E7F83BF0FB681
:1035B000F894A895809160008861809360001092D3
:1035C00060000FBE08950E941E070C94D10282E095
:1035D00084BD93E095BD9AEF97BD80936E000895EA
:1035E0002FB7F89480917E0290917F02A091800283
:1035F000B09181022FBF08952FB7F89460917E0299
:1036000070917F0280918002909181022FBF089576
:103610009C014FB7F89480917E0290917F02A09117
:103620008002B09181024FBF821B930B0895789462
:103630001F920F920FB60F9211248F939F93AF9307
:10364000BF9380917E0290917F02A0918002B09101
:1036500081020196A11DB11D80937E0290937F028D
:10366000A0938002B0938102BF91AF919F918F91FF
:103670000F900FBE0F901F90189587E797E79093D4
:103680000108809300089AE088E10FB6F894A895A5
:10369000809360000FBE90936000FFCF80916F0217
:1036A0000895089522E02093E9002FEF3091E8007B
:1036B000215035FD06C035ED3A95F1F70000211196
:1036C000F5CF2091E80025FF0BC040E050E066E018
:1036D00070E00E94911D8091E8008E778093E80051
:1036E0000895CF93DF9320911801222339F0209180
:1036F000710227FF03C060E222E002C068E021E01F
:103700002093E9002FEF3091E800215035FD06C0ED
:1037100035ED3A95F1F700002111F5CF2091E80041
:1037200025FF1DC0EC0180911801811105C040E00A
:1037300050E068E070E003C070E040E050E0CE018F
:103740000E94911D8091E8008E778093E80080E2CE
:10375000FE01AFE4B2E001900D928A95E1F7DF91AE
:10376000CF91089580934C0270934E0260934D0266
:1037700080918602843001F582E08093E9008FEF2A
:103780009091E800815095FD06C095ED9A95F1F76E
:1037900000008111F5CF8091E80085FF0DC040E069
:1037A00050E063E070E08CE492E00E94911D809113
:1037B000E8008E778093E8000895BC0184E00C94C3
:1037C000B21BBC0183E00C94B21B80918502811175
:1037D00009C00E94221F0E947F1F8091E200846026
:1037E0008093E20008951092850208950C946D1A5A
:1037F0006091820281E0611101C080E00C94581A4E
:103800009091860281E0943009F080E0609182021C
:103810000C945D1A42E061EC81E00E949B1E42E242
:1038200061EC82E00E949B1E9091860281E09430C0
:1038300009F080E0609182020C94661A80918802FF
:10384000833009F461C030F4813071F0823009F4C2
:103850009AC008958A3009F486C08B3009F46CC090
:10386000893009F0A8C020C080918702813A09F010
:10387000A2C08091E800877F8093E80080918B024E
:1038800090918C02892B21F460E28FE492E003C0D6
:1038900060E080E090E070E00E94DC1D8091E80034
:1038A0008B778093E800089580918702813209F038
:1038B00082C080918B0290918C02029708F07BC0AD
:1038C0008091E800877F8093E8008091E80082FD86
:1038D00005C0809186028111F8CF6DC02091F30060
:1038E0008091F20090E0922B029731F48091F100E8
:1038F000813011F0863021F48091F10080936F02C5
:103900008091E8008B7753C080918702813A09F05B
:1039100052C080918B0290918C02892B09F04BC090
:103920008091E800877F8093E8008091E80080FF25
:10393000FCCF8091180136C0809187028132D9F581
:1039400080918B0290918C02892BA9F58091E800DF
:10395000877F8093E8000E94D01E80918902809327
:1039600018010C941E0780918702813221F5809105
:10397000E800877F8093E8000E94D01E80918A0231
:1039800080937002089580918702813AA1F480911A
:10399000E800877F8093E8008091E80080FFFCCFFB
:1039A000809170028093F1008091E8008E7780937F
:1039B000E8000C94D01E089584B7877F84BF0FB6AB
:1039C000F894A895809160008861809360001092BF
:1039D00060000FBE90E080E80FB6F894809361001D
:1039E000909361000FBE0C94681A0E94221F0E94DF
:1039F0007F1FE2EEF0E080818460808378940C94F5
:103A000014228CE091E00C9432198091860285306A
:103A1000A9F480918602853079F40E94B81A8091C9
:103A200084028823B1F30E947A1A882391F30E94BA
:103A30007B1D0E941E07EDCF0C94E31A0895089594
:103A40000C94221D292F332723303105C9F060F44F
:103A50002130310581F02230310509F044C08BE37B
:103A600090E028E732E043C021323105E1F0223214
:103A7000310549F138C082E190E023EB32E037C0F4
:103A800099278130910549F028F0029761F5E0E42B
:103A9000F2E005C0E4E7F2E002C0E2E5F2E0849182
:103AA00090E09F0124C06115710541F061307105FE
:103AB000D1F489E090E023EA32E019C089E090E097
:103AC0002AE832E014C06115710541F061307105DA
:103AD00051F486EB90E025EC32E009C080E490E000
:103AE0002BE733E004C080E090E020E030E0FA0112
:103AF00031832083089580E189BD82E189BD09B4C5
:103B000000FEFDCF8091D8008F7D8093D8008091FA
:103B1000E00082608093E0008091E00081FDFCCFB6
:103B20000895CF92DF92EF92FF920F931F93CF935E
:103B3000DF93EC018B017A010E94EF1E811133C0EB
:103B4000E114F10439F0F70180819181081B190B10
:103B5000C80FD91FC12CD12C0115110519F1809165
:103B6000E80085FD16C08091E8008E778093E8001C
:103B7000E114F10449F0F70180819181C80ED91E4A
:103B8000D182C08285E00FC00E94EF1E882321F3FE
:103B90000AC089918093F10001501109FFEFCF1AFB
:103BA000DF0ADACF80E0DF91CF911F910F91FF9074
:103BB000EF90DF90CF90089520918D0230918E028A
:103BC0002617370748F06115710539F42091E80090
:103BD0002E772093E80001C0B901FC0120E06115B7
:103BE000710579F1809186028823F1F18530F1F138
:103BF0008091E80083FD3CC08091E80082FD2EC0EA
:103C00008091E80080FFEBCF2091F3008091F200DB
:103C100090E0922B6115710551F08830910538F4D0
:103C200021912093F100615071090196F3CF21E0B9
:103C3000089709F020E08091E8008E778093E800F3
:103C4000CECF2111CFCF0AC080918602882361F0A8
:103C5000853061F08091E80083FD0AC08091E80022
:103C600082FFF2CF80E0089582E0089583E0089516
:103C700081E0089520918D0230918E02261737073A
:103C800048F06115710539F42091E8002E772093F2
:103C9000E80001C0B901FC0120E06115710591F156
:103CA00080918602882309F440C0853009F43FC022
:103CB0008091E80083FD3DC08091E80082FD2FC027
:103CC0008091E80080FFE9CF2091F3008091F2001D
:103CD00090E0922B6115710559F08830910540F400
:103CE00024912093F1003196615071090196F2CF31
:103CF00021E0089709F020E08091E8008E7780931A
:103D0000E800CBCF2111CCCF0AC080918602882356
:103D100061F0853061F08091E80083FD0AC08091F8
:103D2000E80082FFF2CF80E0089582E0089583E00A
:103D3000089581E00895982F973068F59093E900F1
:103D4000981739F07091EC002091ED005091F0003F
:103D500003C0242F762F50E021FD02C09F5FECCFDF
:103D60003091EB003E7F3093EB003091ED003D7FD2
:103D70003093ED003091EB0031603093EB007093A5
:103D8000EC002093ED005093F0002091EE0027FD11
:103D9000E5CF80E008958F708093E90081E0089579
:103DA0008091870287FF11C08091E80082FD05C0E5
:103DB000809186028111F8CF11C08091E8008B7745
:103DC0000BC080918602882349F08091E80080FF33
:103DD000F8CF8091E8008E778093E80008952091D5
:103DE000E4003091E50095E64091EC00842F81706D
:103DF00040FF23C08091E80080FD1DC080918602B5
:103E0000882399F0853099F08091EB0085FD11C0F1
:103E10004091E4005091E5002417350729F39150B3
:103E200011F09A01E1CF84E0089582E0089583E0E3
:103E3000089581E0089580E008954091E80042FFF0
:103E4000DDCF08950E94901F0E94981FE0EEF0E0E1
:103E5000808181608083E8EDF0E080818F778083CE
:103E600019BCA7EDB0E08C918E7F8C9380818F7E02
:103E700080831092850208950F931F93CF93DF9351
:103E80000E94901F0E94981FC8EDD0E088818F7714
:103E9000888388818068888388818F7D888319BC26
:103EA0001092860210928202109284021092830273
:103EB00000EE10E0F80180818B7F80838881816033
:103EC000888342E060E080E00E949B1EE1EEF0E02B
:103ED00080818E7F8083E2EEF0E08081816080834C
:103EE000808188608083F80180818E7F80838881D3
:103EF00080618883DF91CF911F910F910895E8ED44
:103F0000F0E080818F7E8083E7EDF0E0808181604A
:103F1000808384E082BF81E0809385020C943C1F03
:103F2000E8EDF0E080818E7F80831092E2000895BA
:103F30001092DA001092E10008951F920F920FB6CE
:103F40000F9211242F933F934F935F936F937F931F
:103F50008F939F93AF93BF93EF93FF938091E10073
:103F600082FF0BC08091E20082FF07C08091E100D8
:103F70008B7F8093E1000E9413228091DA0080FF02
:103F80001FC08091D80080FF1BC08091DA008E7F17
:103F90008093DA008091D90080FF0DC080E189BD57
:103FA00082E189BD09B400FEFDCF81E080938602E5
:103FB0000E94E51B05C019BC109286020E94F31BEB
:103FC0008091E10080FF19C08091E20080FF15C060
:103FD0008091E2008E7F8093E2008091E200806118
:103FE0008093E2008091D80080628093D80019BC51
:103FF00085E0809386020E94F81B8091E10084FF97
:1040000030C08091E20084FF2CC080E189BD82E154
:1040100089BD09B400FEFDCF8091D8008F7D8093CB
:10402000D8008091E1008F7E8093E1008091E200D2
:104030008F7E8093E2008091E20081608093E200B5
:1040400080918202882311F084E007C08091E30010
:1040500087FD02C081E001C083E0809386020E9458
:10406000001C8091E10083FF29C08091E20083FF62
:1040700025C08091E100877F8093E10082E08093FA
:104080008602109282028091E1008E7F8093E1008F
:104090008091E2008E7F8093E2008091E200806157
:1040A0008093E20042E060E080E00E949B1E8091ED
:1040B000F00088608093F0000E94F61BFF91EF9162
:1040C000BF91AF919F918F917F916F915F914F9130
:1040D0003F912F910F900FBE0F901F9018951F9238
:1040E0000F920FB60F9211242F933F934F935F932C
:1040F0006F937F938F939F93AF93BF93CF93DF93F0
:10410000EF93FF93C091E900CF708091EC00D82F1E
:10411000D17080FDD0E81092E9008091F000877F97
:104120008093F00078940E94B3201092E90080916F
:10413000F00088608093F000CD2BCF70C093E90031
:10414000FF91EF91DF91CF91BF91AF919F918F91AF
:104150007F916F915F914F913F912F910F900FBE83
:104160000F901F9018951F93CF93DF93CDB7DEB7B5
:10417000AA970FB6F894DEBF0FBECDBFE7E8F2E016
:104180008091F100819322E0EF38F207C9F70E9495
:104190001E1C8091E80083FF2EC1809187029091C0
:1041A0008802492F50E04A30510508F024C1FA0135
:1041B000EE59FF4F0C948922803821F0823809F0A3
:1041C0001AC108C08091830290918402992389F0DA
:1041D00082600FC080918B028F70873008F00BC116
:1041E0008093E9008091EB0085FB882780F910928D
:1041F000E9009091E800977F9093E8008093F100A8
:104200001092F100D1C0282F2D7F09F0F4C088232F
:1042100019F0823061F0EFC080918902813009F09D
:10422000EAC0933009F080E0809384022EC0809130
:10423000890281112AC080918B028F702FEF280F85
:10424000263008F0D8C08093E9002091EB0020FFD1
:104250001CC0933021F48091EB00806214C09091D7
:10426000EB0090619093EB0021E030E0A90102C0E7
:10427000440F551F8A95E2F74093EA001092EA0036
:104280008091EB0088608093EB001092E9008091B0
:10429000E800877F8093E8000E94D01EACC08111A7
:1042A000AAC0109189021F778091E3008078812B4A
:1042B0008093E3008091E800877F8093E8000E946C
:1042C000D01E8091E80080FFFCCF8091E3008068E1
:1042D0008093E300111102C082E001C083E080936B
:1042E000860289C08058823008F085C0809189029A
:1042F00090918A028C3D53E0950779F583E08A839B
:104300008AE289834FB7F894DE01139620E03EE0FD
:1043100051E2E32FF0E050935700E49120FF03C0F7
:10432000E295EF703F5FEF708E2F90E0EA3010F073
:10433000C79601C0C0968D939D932F5F243149F796
:104340004FBF8091E800877F8093E8006AE270E0C9
:10435000CE0101960E94DC1D16C060918B02709107
:104360008C02AE014F5F5F4F0E94201DBC01892B64
:1043700009F441C09091E800977F9093E80089810B
:104380009A810E943A1E8091E8008B778093E80022
:1043900032C0803881F58091E800877F8093E80003
:1043A000809182028093F1008091E8008E7772CF35
:1043B000811121C08091890290918A0299270297E8
:1043C000D4F48091E800877F8093E800809189028F
:1043D000809382020E94D01E80918202811106C0C9
:1043E0008091E30087FD02C081E001C084E08093FA
:1043F00086020E940A1C8091E80083FF0AC0809117
:10440000E800877F8093E8008091EB0080628093D2
:10441000EB00AA960FB6F894DEBF0FBECDBFDF91BA
:10442000CF911F9108950895CF938091860288239C
:10443000A1F0C091E900CF709091EC00892F8170BC
:1044400090FD80E8C82B1092E9008091E80083FD80
:104450000E94B320CF70C093E900CF910895DB0193
:104460008F939F930E949E22BF91AF91A29F800D38
:10447000911DA39F900DB29F900D11240895AA1B2A
:10448000BB1B51E107C0AA1FBB1FA617B70710F03F
:10449000A61BB70B881F991F5A95A9F78095909571
:1044A000BC01CD01089597FB072E16F4009407D0A8
:1044B00077FD09D00E943F2207FC05D03EF490957D
:1044C00081959F4F0895709561957F4F0895A1E262
:1044D0001A2EAA1BBB1BFD010DC0AA1FBB1FEE1F7E
:1044E000FF1FA217B307E407F50720F0A21BB30BC9
:1044F000E40BF50B661F771F881F991F1A9469F745
:1045000060957095809590959B01AC01BD01CF01A0
:104510000895EE0FFF1F0590F491E02D0994A29FDE
:10452000B001B39FC001A39F700D811D1124911D87
:10453000B29F700D811D1124911D08950E948F223C
:10454000A59F900DB49F900DA49F800D911D1124E7
:104550000895FB01DC0104C08D910190801921F4C4
:1045600041505040C8F7881B990B0895F999FECF28
:1045700092BD81BDF89A992780B50895A8E1B0E071
:1045800042E050E00C94EA22262FF999FECF92BD2A
:1045900081BDF89A019700B4021639F01FBA20BD08
:1045A0000FB6F894FA9AF99A0FBE08950396272F3A
:1045B0000E94C5220E94C422252F0E94C522242FBA
:1045C0000C94C5220196272F0E94C5220C94C42268
:1045D000DC01CB01FC01F999FECF06C0F2BDE1BDC3
:1045E000F89A319600B40D9241505040B8F70895B2
:0445F000F894FFCF6D
:1045F400C8000002280850011E0A14014E1B711B3A
:10460400521BE11BDD1B511B01E200E900EA00B56E
:1046140000B600B700CD008301CC008A019201945A
:10462400012102230224022502260227022A02B3C0
:1046340000B4006F007000818283E200E900EA00A8
:10464400B500B600B700CD008301CC008A01920109
:1046540094012102230224022502260227022A02AF
:10466400B300B4006F00700081828334C6976694EF
:0646740090F731333236ED
:00000001FF
